S023000052414D436F646556325F4C504331314178785F454550524F4D5F4C452E6D6F7493
S1130000D100F9010102150233026F0295020000CA
S1130010F7B582B01C00A44D8020C004A860A34F93
S1130020402003998906890E401A0499884201D216
S1130030009000E000910A98C0070DD503987860FD
S113004008203860029800F025F928684001F9D5A5
S11300508020C004A86003E000207860032038609A
S1130060009E0A98C00702D5F868207001E0207845
S1130070B8600A98800700D4641C029800F00AF95A
S113008028684001F9D58020C004A860761EE8D114
S11300900A98C0070FD480204005A86003987860B0
S11300A006203860029800F0F5F82868C000F9D5F9
S11300B080204005A86004980099401A0490039891
S11300C000994018039004980028A9D105B0F0BD08
S11300D0F0B583B0040050680600E16B002901D03C
S11300E00D4671E0019072480068A0617048806814
S11300F0E0616F48006920626E4F38686062B86FD3
S1130100A062786FE0626A48016041600121416049
S11301108160206A18210143654801613B203860F1
S11301202020B86764487867644820636448606343
S11301306448A06301200090019B4022002120001C
S1130140FFF766FF00200090230030334022002197
S11301502000FFF75DFFFD0C0120009023003033E9
S11301600C2229002000FFF753FF206B53498842DB
S11301700BD1606B5249884207D1A06B5149884228
S113018003D16D08780D8542E6D26D09402D00D16A
S11301903F2500200090019B402200212000FFF712
S11301A037FF4348E1698160A06941490860084616
S11301B00021416001214160216A0161606A386067
S11301C0A06AB867E06A7867002030800620B070C3
S11301D00120F070307170710020B071F0713072D4
S11301E070720120B0723061002070614020F061B3
S11301F0B561E56303B0F0BD80B51100012202E0F2
S113020080B51100002200924B684A690969FFF722
S1130210FFFE01BD00B583B011000022D24301925C
S11302200222009201AB40220969FFF7F1FE03B0FC
S113023000BD1F490A6802608A6842600A698260D8
S1130240182313430B6100220A604A6001224A60AA
S11302508A6018490A68C2608A6F02614A6F426103
S11302603B2008602020886713484867704710497E
S113027042688A6002680A6000224A6001224A6079
S113028082680A610B49C2680A6002698A67406928
S1130290486770470C480168C90703D5AA218160E3
S11302A05521816070470000E0CF034080C00340C7
S11302B0708004401CC003400F0F0F00416C657830
S10F02C04375737454657374004000406F
S9030000FC
